:020000040000FA
:02000000552980
:100008007E1480312000111CA428CE01CD01E730D8
:1000180097009630960011100130E002031D1A284F
:100028000130F7060A30F5007508E0006A26F50089
:1000380075082000C200420803192B2842088600D0
:100048008701403FA000413FA100423FA200200895
:1000580003194E28A01D3228771C4E28073020058A
:10006800F50002307506031D4928E030840087300A
:1000780085001200023A031943280230442805304B
:10008800C3000030C40043084B2820080739F50096
:100098007508CD04210803197128A11D5528771C5E
:1000A800712807302105F50002307506031D6C28FC
:1000B800E0308400873085001200023A0319662870
:1000C800023067280530C5000030C60045086E2894
:1000D80021080739F5007508CE040310CE0D03106A
:1000E800CE0D0310CE0D220803199A28A21D7E28D2
:1000F800771C9A2807302205F50002307506031D83
:100108009528E0308400873085001200023A0319F0
:100118008F28023090280530C7000030C8004708F3
:10012800972822080739F5007508CE048C1FA028E7
:100138004E098C004D09A3284E088C004D088E00EE
:10014800911C53299110CF010330F5007508F00078
:100158004F08CD262B3EF60076082000D000F12867
:100168000E08F5000630F536890BB7287508F60035
:100178007608A900901929158E1DC7282908FD3E63
:1001880084008630E0280C1BCB280530CC280730AB
:10019800C9000030CA000E1AD3280330D42807300B
:1001A800CB000030CC004B084905F5007508A905BF
:1001B8002908F53E840086300318013E85000008B2
:1001C800E6280D08F5007508EF2803108E1E0314A5
:1001D800003003180130A90004294F08F500F60182
:1001E8007608003A0319F92804297508003A031912
:1001F800B428013A0319E528033A0319E928042920
:1002080050088600870101082906031D1129500896
:10021800023E8600870181014B295008023E860074
:100228008701010803193029500A8600870101084F
:100238002906031D30295008023E86008701013037
:100248008102031D4B292908F50050088600870103
:1002580075088100F7144B292908F500500A860013
:10026800870175088100E130840087308500000827
:10027800F5000130F535FF3E031D3E297535043E76
:10028800F6005008023E860087017608810001309A
:10029800F5007508CF0703304F02031CA8287E100D
:1002A800090056290B27DD000C27DE000D27DF008B
:1002B8000E27E000F701F8012030840000308500A7
:1002C80022300527A0308400003085001230052731
:1002D8007E102000EF2A003400340034003400344B
:1002E8000034003400340034003400340034003466
:1002F8000034003400340034003400340034003456
:1003080000340034003401340A340A3401340A3425
:100318000A3401340A340A3401340A340A34013400
:100328000A34043401340A34043401340A340C34F1
:10033800013401340434003400340034003400340F
:100348000034003400340034003400340034003405
:1003580000340034003400340034003400340034F5
:1003680000340034003401340A340A3401340A34C5
:100378000A3401340A340A3401340A340A340134A0
:100388000A34043401340A34043401340A340C3491
:1003980001340134043400340034003400340034AF
:1003A80000340034003400340034003400340034A5
:1003B8000034003400340034003400340034003495
:1003C80000340034003401340A340A3401340A3465
:1003D8000A3401340A340A3401340A340A34013440
:1003E8000A34043401340A34043401340A340C3431
:1003F800013401340434003400340034003400344F
:100408000034003400340034003400340034003444
:100418000034003400340034003400340034003434
:1004280000340034003401340A340A3401340A3404
:100438000A3401340A340A3401340A340A340134DF
:100448000A34043401340A34043401340A340C34D0
:1004580001340134043401340234093401340234DF
:1004680009340134023409340134023409340134C2
:1004780002340934013402340934013402340934B1
:10048800013402340934013404340A3401340434A4
:100498000A34013404340A34013404340A3401348B
:1004A80004340434013404340434013404340C3482
:1004B800013404340134013402340934013402347F
:1004C8000934013402340934013402340934013462
:1004D8000234093401340234093401340234093451
:1004E800013402340934013404340A340134043444
:1004F8000A34013404340A34013404340A3401342B
:1005080004340434013404340434013404340C3421
:1005180001340434013401340A34093401340A340E
:10052800093401340A34093401340A3409340134F1
:100538000A34093401340A34093401340A340934D8
:1005480001340A34093401340C340A3401340C34CB
:100558000A3401340C340A3401340C340A340134BA
:100568000C34043401340C34043401340C340C34A9
:1005780001340C34013402340134093402340134B6
:1005880009340234013409340234013409340234A0
:100598000134093402340134093402340134093491
:1005A800023401340934023402340134023402348E
:1005B8000134023402340134023402340134023486
:1005C8000434013402340434013402340C34013468
:1005D80004340134013448302100950089252D2444
:1005E800F71CF42AF710702B2000BF01BE01BD01D3
:1005F800882B01303D3E8600870102303D3E840055
:1006080085010130803FC03F3E2B20002E0821008D
:10061800B60036082000DC00DC1F432B5C087F395D
:100628002100B600B70136082000D10021003708A4
:100638002000D2000330D3000030D4008B262000E5
:1006480052088500510884006F3084078130853D49
:10065800003FBD00013FBE00023FBF003108031943
:10066800882BF8302E052100B600F8303606031D19
:10067800882B0A30B60036082000BD00882B5D089C
:10068800BD005E08BE005F086E2B20002E0821000A
:10069800B6000430B636890B4E2B3608B700B801C1
:1006A80037082000D100210038082000D20003308C
:1006B800D3000030D4008B26200052088500510852
:1006C8008400BE3084078530853D003FBD00013F72
:1006D800BE00023FBF00882B20002B082100B60077
:1006E800B7013708003A03197A2B882B3608003AE5
:1006F8000319F82A013A0319FD2A033A0319492B69
:10070800063A0319092B882BE030840087308500CE
:1007180012000319D22B20003D08B7003E08B8008C
:100728003F08B9003D082100B60036082000D10076
:1007380023084726003A0319A62B2000B701B70A59
:10074800AA01AA0A20003E082100B60036082000A7
:10075800D10024084726003A0319B72B2000B80116
:10076800B80AAA01AA0A20003F082100B6003608E4
:100778002000D10025084726003A0319C82B20007D
:10078800B901B90AAA01AA0A20002A080319162CD5
:100798003730EE253D30EE253730152C2000230864
:1007A8003D060319DB2B2100B901BA01E32B23080D
:1007B8002100B600B7013608B9003708BA00390871
:1007C800B60036082000BA0024083E060319F02BAC
:1007D8002100BB01BC01F82B24082100B600B70199
:1007E8003608BB003708BC003B08B60036082000B6
:1007F800BB0025083F060319052C2100BD01BE01D9
:100808000D2C25082100B600B7013608BD003708B1
:10081800BE003D08B60036082000BC003A30EE2580
:100828003A30EE25200023083D06031D232C24081A
:100838003E06031D232C25083F060319F42A3D30E4
:10084800EE2520003D08A3003E08A4003F08A500AF
:10085800F42A0130A7261E26003A03197C2C200012
:10086800A6012608E03E840087300318013E850073
:100878000008D9002608403E8600870159088100F3
:100888000130D9005908A60702302602031C352C6E
:100898001E26003A031D4C2C20000C1B612C0D0851
:1008A800D9005908A600A60EA60C0730A6052608EA
:1008B800073CD9005908C1006E2C8D1B652CC0015E
:1008C8006E2C0D1B6A2CC001C00A6E2C0230D90098
:1008D8005908C000E030D1000730D2004030D900BC
:1008E8005908D3000230D4000030D5004025C22C6E
:1008F80020008C1B832C2100B201B301882CFF300F
:100908002100B2000030B300320820008E008C00B5
:1009180006302000DA001330D900AD30890B922C54
:10092800D90B922CDA0B922C00320030DE26D03E06
:10093800C5240230DE26D03EC5240330DE26D03E54
:10094800C52420008C1BAC2C2100B401B501B12CAE
:10095800FF302100B4000030B500340820008E00BC
:100968008C0004302000DA008E30D9001230890B58
:10097800BB2CD90BBB2CDA0BBB2C00000030A726F4
:1009880008002000D3005308031D022D092D8C1BDD
:10099800D02C20000C14D22C20000C100C1CD72CAE
:1009A80020000E14D92C20000E1002302000D20096
:1009B8000430D100BA30890BDF2CD10BDF2CD20BDD
:1009C800DF2C000020008C1FEC2C20000C14EE2CD7
:1009D80020000C100C1CF32C20000E14F52C200009
:1009E8000E1002302000D2000430D100BA30890B3A
:1009F800FB2CD10BFB2CD20BFB2C00000130200070
:100A0800D302530A0319332DCB2C8C1B0E2D200037
:100A18000C14102D20000C100C1C152D20000E1489
:100A2800172D20000E1007302000D2001730D100FB
:100A38006A30890B1D2DD10B1D2DD20B1D2D0000E9
:100A480020008C1F2A2D20000C142C2D20000C10A7
:100A58000C1C312D20000E14332D20000E100530F3
:100A68002000D2000F30D100F130890B392DD10B85
:100A7800392DD20B392D0800200051082300910090
:100A88002000520823009200151315161515EC26A0
:100A9800230015111512951615152000520823006C
:100AA80092002000D8015508803A803C031D5E2D35
:100AB800540858020318862D2000510858072300AF
:100AC8009100200058085307D60056088600870171
:100AD8000108230093003430940020005408FF3E9E
:100AE800D600FF30553DD700580856065704031D59
:100AF8007F2D23009512EC2601302000D6005608E1
:100B0800D807572D230015110800683021009900D7
:100B180020008C1B922DD101D201962DFF30D100DF
:100B28000030D20051088E008C00C03021008C00AB
:100B3800FF308D00F8308E00FF309000FF30240029
:100B48008D0023008C018D018E01270094018B01FB
:100B5800313020009800E7309700963096004E30EC
:100B68009C00C8309B00F7102100111491148B17BA
:100B78000B17080001340134023401340134023403
:100B880001340134023401340134023401340134B3
:100B980002340134013402340134013402340134A2
:100BA80001340234013401340A34013401340A3482
:100BB800013401340A34013401340A340134023472
:100BC800013401340234013401340A34013402346A
:100BD800013401342000D9002708D5005508DA006F
:100BE8000130D5005508DA0706305A020318DA0131
:100BF8005A0828060319FC2D590886008701403F2A
:100C0800D500413FD600423FD7000330D8005808EE
:100C1800D1002708BB26A03E860087012000550882
:100C2800C03F5608C13F5708C23F5A08D50055086B
:100C3800A700080020000E1027302000D100F53052
:100C4800890B242ED10B242E20008E1C2D2E003033
:100C580008000E1427302000D100F530890B322E01
:100C6800D10B322E20008E1C2B2E0E102730200088
:100C7800D100F530890B3E2ED10B3E2E20008E1868
:100C88002B2E013008002000D30007305305D20076
:100C980004305206031D612E07305105D200023080
:100CA800520603195F2E612E07305105D200043019
:100CB8005206031D682E0130080007305305D20084
:100CC800023052060319582E003008002000280868
:100CD8002706031D712E003008000330F400740845
:100CE800F0002808CD26A03E86008701403F20005E
:100CF800B400413FB500423FB6000130F40074082B
:100D0800A807063028020318A8013430080020007C
:100D1800D501D601511C942E5308D5075408D63D49
:100D28000130D335D40D890B952E0130D236D10C34
:100D3800890B9A2E51085204031D8E2E5608D20094
:100D48005508D10008002000D20052080319B22E1D
:100D58000F272000181021008E140800FD30D10044
:100D6800510821008E05200018148B170800200058
:100D7800D400D301541CC42E5108D2005208D30702
:100D88000310D10D0310D40C5408031DBE2E5308B4
:100D98000800F200F301721CD52E7008F1007108EA
:100DA800F3070310F00D0310F20C7208031DCF2E89
:100DB800730808002000D1005108230091008030FA
:100DC80092001517151400000000230013080800EE
:100DD800553023009600AA309600951400000000B4
:100DE800080001340134013401340234003404347D
:100DF8000034003400340234013400340234043442
:100E08000034640080010131890B062F003401345D
:0E0E1800013402340A348B138B1F0800102F94
:100FC000023400340034003400340034003400347F
:100FD0000034003400340034003400340034003471
:100FE0000034003400340034003400340034003461
:100FF0000034003400340034003400340034003451
:020000040001F9
:0800000033002E003100310035
:04000E00A4C9FFD5AD
:00000001FF
